:10000000000C2500400C26000F0C0500B30C060068
:10001000280C020045077C0AE6074A0B06075F0A20
:100020000F0C05006500000C3800000C3900010CB5
:100030003A00020C3B00030C3C00060C3D00070C90
:100040003E00000C3F000102320006023000730047
:1000500074000102370092014306290A1702320098
:10006000B302060237009001200E43063E0A070C39
:100070007301180CD3012400000233001702300072
:100080001302070E040F43074E0A1702B4010602BB
:10009000F70EB407080D2600170234000602BF0E43
:1000A0005307400D26000F0C5307FD0E05000400FA
:1000B00006070A0AE6070A0A45070A0A290A0F0C70
:1000C00005006500070C41014307620A0F0C05009B
:1000D00026066D0A0602040F2600070C4101040FD4
:1000E00043076D0A0D0C0500040006060A0AE60720
:1000F0000A0A45070A0A620A0607340B0F0C0500B4
:100100006500010232000602300073007400110520
:10011000200C350001078A0A6100C605FF0CF501B5
:1001200006023700B707980AB006980A120CF501C4
:1001300017023000070C1106080D050001079E0A82
:10014000610006023700B707AC0AB006AC0AFF0C24
:10015000F5010107A90A610017023000200C950083
:100160000307B5000107B20A610006023700B707AE
:10017000C00AB006C00AFE0CF5010107BD0A610005
:1001800017023000600C95000306B5000107C60A8F
:10019000610006023700B707D40AB006D40AFE0C85
:1001A000F5010107D10A6100170230001107DC0ACE
:1001B000450C9500030611040107DC0A61000602E4
:1001C0003700B707EA0AB006EA0AFE0CF501010794
:1001D000E70A610017023000B401F70EB407080DFA
:1001E000260017023400C6040107F40A6100040067
:1001F0001106FE0A250C95000307110506023700BB
:10020000B707090BB006090BFE0CF5011702300009
:100210001B0B1702300001070B0B610006023700B1
:10022000B707190BB006190BFE0CF50117023000C9
:100230002F0B1702300001071B0B6100060237006D
:10024000B7072D0BB0062D0BFF0CF5011702300080
:1002500006070A0A45060A0A8D0A17023000060731
:100260000A0A45060A0A8A0A0F0C0500650073008F
:100270000502310025063A0BB3022606420B0602A0
:10028000040F26002507420B040006060A0A45064D
:100290000A0A3A0B06076D0B0F0C0500650086076E
:1002A0004F0BC6050F0C0500220C370086075E0BAE
:1002B0000507660405066605F702560BC604070C1B
:1002C0003700F702610B0D0C0500040006070A0A4F
:1002D000E6060A0A45070A0A4F0B0F0C05006500DF
:1002E0008606700B0E0C0500400C370086067A0B54
:1002F000F702760B0D0C0500000000000000000066
:100300000D0C2607FE0E0500040006060A0AE60686
:0A0310000A0A45070A0A700B0A0AE0
:0203FE00000AF3
:0804000003000A0000000300E4
:00000001FF
